:1000000004308A00922C00001F1555101F1D551436
:1000100055180E2855101F1D551408281F190E2895
:100020001E08FA0083161E088312D6001E08D70089
:100030005608F8005708F9000800520DF700F70DB0
:10004000F70DF830F7051F08C73977049F0009300E
:10005000F700F70B29282C280420790808005230D3
:10006000840083130008031942280230F800F701C6
:10007000F70B3828F80B37289730F700F70B3E2896
:10008000800B3528080004207908D3007808D200B6
:1000900004207908FA007808D20779080318790F44
:1000A000D30704207908FA007808D20779080318E2
:1000B000790FD30704207808D20779080318790F3D
:1000C000D307530CFA00520CF900FA0CF90C3F302C
:1000D000FA057908F8007A08F90008004D08D200FE
:1000E0001D20CF01CE014E08133C031C8A2843205B
:1000F0007908D1007808D000D108031D8528500860
:10010000043C031C85280130CF000130D2002F2091
:10011000CE0A73284F08F80008001030D100F7010C
:10012000FA01CE0CCD0C031C9B284F08F7070318CF
:10013000FA0A5008FA07FA0CF70CF90CF80CD10B74
:1001400091280800F801F901F701FA015008031D90
:10015000AC284F080319C6281030D1000310CD0D6C
:10016000CE0DF70DFA0D50087A02031DB9284F087D
:100170007702031CC2284F08F702031CFA03500839
:10018000FA020314F80DF90DD10BAE28080008305F
:10019000CE02031CD7284E30840083130310800C3A
:1001A00000080319D728D5280000800BD4280800A0
:1001B0000612A701073083168600811325308500BB
:1001C0001F1383121F139F1783169F1783121F1469
:1001D00083161F109F141F159F158312D2011D2017
:1001E0000619FA280630C000FA30D2002F20C00BC2
:1001F000F42801290C30C000FA30D2002F20C00BA7
:10020000FC28CD016E207808A00006160130A7005A
:100210006430D2002F2043207908A2007808A10082
:10022000861843292208CE002108CD00D0011330C2
:10023000CF008D207908A4007808A3002408CE0000
:100240002308CD00D0011430CF00A2207908A400EB
:100250007808A3002208CE002108CD00D001273065
:10026000CF008D207908A6007808A5002608CE00CA
:100270002508CD00D0012830CF00A2207908A600A3
:100280007808A50073292208CE002108CD00D001EE
:100290001130CF008D207908A4007808A30024082D
:1002A000CE002308CD00D0011430CF00A220790861
:1002B000A4007808A3002208CE002108CD00D001B8
:1002C0002530CF008D207908A6007808A5002608E3
:1002D000CE002508CD00D0012830CF00A22079081B
:1002E000A6007808A500A008031DC529BC01BB0114
:1002F00043207908B8007808B70038082402031CA6
:100300008B29031D87292308370203188B2906121E
:10031000A701BC01BB010618BA29A708031DBA2909
:1003200026083802031C9E29031D9A293708250236
:1003300003189E29BB0A0319BC0AA029BC01BB01F2
:100340000619AD293B08DC3C031DAD293C08053CE2
:10035000031DAD2906160130A700061DBA293B086A
:10036000B83C031DBA293C080B3C031DBA290616EC
:100370000130A7000530C0009030CE00C720C00B70
:10038000BC298616861278291D2A04207908BA000D
:100390007808B9001430BF00BE01BD0143207908C0
:1003A000B8007808B700B808031DDA293708323CCE
:1003B0000318DD291430BF00E029BF08031DBF0367
:1003C000BF08031DE7290612BE01BD01A7010618DB
:1003D000132AA708031D132ABF080319F329BD0A0E
:1003E0000319BE0AF529BE01BD010619042A3D08FC
:1003F000DC3C031D042A3E08053C031D042A0616A6
:100400000130A700BE01BD01061D132A3D08B83CFE
:10041000031D132A3E080B3C031D132A0616013048
:10042000A700BE01BD010530C0009030CE00C7203E
:10043000C00B152A86128616CE29AE2C4D0DF7005C
:10044000F70DF70DF830F7051F08C73977049F003F
:100450000930F700F70B2A2A2D2A04207908CF004B
:100460007808CE0004207908FA007808CE077908C9
:100470000318790FCF0704207908FA007808CE070F
:1004800079080318790FCF0704207808CE07790878
:100490000318790FCF074F0CFA004E0CF900FA0C35
:1004A000F90C3F30FA057908F8007A08F9000800DD
:1004B0000230D2001D207808AD0779080318790FA3
:1004C000AE07003003180130AF07003003180130C9
:1004D000B0070330D2001D207808B107790803184F
:1004E000790FB207003003180130B307003003184A
:1004F0000130B407B50A0319B60AB508031DE52A89
:100500003608043C031DE52AD501300CD4002F0C1D
:10051000D3002E0CD200D40CD30CD20C3F30D40517
:100520005208CD0053080339CE00D501340CD40055
:10053000330CD300320CD200D40CD30CD20C3F308D
:10054000D4055208CF0053080339D0004E08013CAF
:100550000318B12AFF3A031DD02A4D08653C031C3D
:10056000D02A4E08013C031CBB2A031DD02A4D088B
:10057000993C0318D02A5008013C0318C62AFF3AB8
:10058000031DD02A4F08653C031CD02A5008013CAB
:10059000031CD62A031DD02A4F08993C031CD62AD7
:1005A00006148619D52A86136300D72A0610B601C9
:1005B000B501B401B301B201B1013408B000330890
:1005C000AF003208AE003108AD0008008613A70165
:1005D0007C308316860083120610861083168113E2
:1005E0003F3085001F1383121F139F1783169F1719
:1005F00083121F1483161F109F101F119F110230AA
:100600008312AB00AA012B08A9002A08A800193000
:10061000AC00061B132B0630CD00FA30D2002F2081
:10062000CD0B0D2B1A2B0C30CD00FA30D2002F2021
:10063000CD0B152B0130CD006E207808A000861759
:100640000130A7006430D2002F2043207908A20097
:100650007808A100861A5D2B2208CE002108CD0063
:10066000D0011230CF008D207908A4007808A300B3
:100670002408CE002308CD00D0011430CF00A220E2
:100680007908A4007808A3002208CE002108CD0034
:10069000D0011330CF008D207908A6007808A5007E
:1006A0002608CE002508CD00D0011430CF00A220AE
:1006B0007908A6007808A5008D2B2208CE00210815
:1006C000CD00D0010E30CF008D207908A40078082D
:1006D000A3002408CE002308CD00D0011430CF00A1
:1006E000A2207908A4007808A3002208CE002108DF
:1006F000CD00D0011130CF008D207908A6007808F8
:10070000A5002608CE002508CD00D0011430CF006A
:10071000A2207908A6007808A500B401B301B201AF
:10072000B1013408B0003308AF003208AE00310820
:10073000AD00B601B501A008031D342CBC01BB01FE
:100740000130CD001E227908B8007808B700061DD8
:10075000AC2B0030F800E62BCD011E227908A90051
:100760007808A8002A082802CD002908CE002B0806
:10077000031C2B0FCE02CE08031DC22B4D08053CD7
:100780000318C92B1630AC002908AB002808AA00B2
:10079000D72B29082B02031CD72B031DD32B2A0888
:1007A00028020318D72B2908AB002808AA00AC0898
:1007B000031DAC03AC080319E22B86140130F800CA
:1007C000E62BE62B86100030F800E62B7808CC00EC
:1007D00038082402031CF92B031DF22B23083702CF
:1007E0000318F92BCC08031DF92B8613A701BC01B4
:1007F000BB01061A2B2CA708031D2B2C2608380238
:10080000031C082C031D0B2C37082502031C0B2C82
:10081000CC0803190F2CBB0A0319BC0A112CBC010C
:10082000BB01061B1E2C3B08DC3C031D1E2C3C0898
:10083000053C031D1E2C86170130A700061F2B2C1C
:100840003B08B83C031D2B2C3C080B3C031D2B2CF8
:1008500086170130A70058229930F700F70B2E2C8D
:1008600005170513A02B912C0130D2001D2079080B
:10087000BA007808B9001430CB00BE01BD010130C8
:10088000CD001E227908B8007808B700B808031D0B
:100890004D2C3708323C0318502C1430CB00532C0D
:1008A000CB08031DCB03CB08031D5A2C8613BE01B6
:1008B000BD01A701061A862CA708031D862CCB08AC
:1008C0000319662CBD0A0319BE0A682CBE01BD01BE
:1008D000061B772C3D08DC3C031D772C3E08053CAD
:1008E000031D772C86170130A700BE01BD01061F2E
:1008F000862C3D08B83C031D862C3E080B3C031D8E
:10090000862C86170130A700BE01BD015822033096
:10091000CD00B330CE00C720CD0B892C05130517B1
:100920003F2CAE2C840183131F3083057030831657
:100930008F000F081F149F141F159F11FF30850093
:100940008312051DA72C851AA72CD828AE2C051AB2
:0E095000AD2C851EAD2CE62AAE2C6300630094
:02400E00501F41
:00000001FF
